:020000040000FA
:1000000077289818181218162C08A0002D08A1009F
:10001000A201A3010B280C2864008C1A2828FF30A9
:10002000A207031CA307031CA007031CA107031CB2
:100030000800220F0A28230F0B286430A20000308A
:10004000A3000C2898181812181664008C1E252876
:100050001A080314722864000C1E2B28990003143C
:100060007228A40029080314031972286D20031CA8
:100070000800A000251883172408840020088000A9
:100080008313A40AA9033228A301A200FF30A20708
:10009000031CA307031C72280330A100E330522085
:1000A0004628A101F43EA000A109FE30031C5B28F4
:1000B000A00703185828A0076400A10F58280000C3
:1000C000201862282018642808000310A00DA10D34
:1000D000FF3E0318652820087228840031088A0032
:1000E0003008820083130313831264000800831610
:1000F0000C309900203098008312903098008A11BB
:10010000EF2983120313F80194013E309400831603
:10011000031306168614831203138C11080083122E
:100120000313FF30FF00F70083120313F70B9D2822
:10013000FF0B9D280530E021B62883160313141AFF
:10014000A32894199428831203133A308400B12110
:100150007818B62878100008FD0056217818B628BF
:10016000840AF60BAB28C721781CBA287A08F50058
:100170007810E629080083120313FF30FF00F70010
:1001800083120313F70BC928FF0BC9280530E021A0
:100190000E2983160313141ACF289419C02883122A
:1001A00003133A308400FA2883120313FF30FF0050
:1001B000F70083120313F70BE228FF0BE228053048
:1001C000E0210E2983160313141AE8289419D9285C
:1001D000831203133A308400B12178180E290008E5
:1001E000FD00562178180E293B08FD00562178188D
:1001F0000E29C721B12178180E290008FD007D14B1
:10020000562178180E29422178180E29840A7E0872
:100210008000F60B0329C721781C12297A08F50003
:100220007810E629080083120313FF30FF00F7005F
:1002300083120313F70B2129FF0B21290530E0213D
:100240003D2983160313141A272994191829831298
:1002500003133A308400B12178183D290008FD00CD
:100260007D14562178183D29422178183D29840AA9
:100270007E088000C721781C41297A08F500781093
:10028000E62908000830FF00FE01FE0D031C7E1069
:1002900003187E146C21F91B7E14FF0B4529760888
:1002A000FF007917FF0B7913872100340830FF0016
:1002B0007913FD1B791787217818E0217818E62932
:1002C000FD0D031C7D1003187D14FF0B58296C21B4
:1002D0000330F91BE02100348316031386148312C4
:1002E0000313F91383160313061683120313061A56
:1002F0007A297729861C7D29F91700000000000063
:100300000000831603130612831203130034791FAF
:10031000952983160313861402308312031386185B
:100320009B29781CFA0078149B29831603138610E6
:1003300000000000000083160313061600000000F2
:100340000000013083120313061AA729A429000014
:10035000000000000000831603130612831203132B
:100360000034831603138614061683120313000049
:10037000000000000130061EE021831603138610E2
:1003800000000000000006128312031300348316DD
:1003900003138610061683120313000000000000EA
:1003A00000000000000000000000061ED529831692
:1003B000031386140430861CE021831203130034D7
:1003C00083120313781CFA0078140034861406167E
:1003D0008316031386140616831203130034831640
:1003E00070308F0007309C009B01810183128A01CD
:1003F00081208A11C0238A0181208A01222083164C
:10040000A200640022087E3C8A118312031D0A2A7E
:100410008A110C228A01FD29E830AC000330AD00BE
:100420008A0101208A11031C402C8316A300831229
:100430008A0101208A11031C402C8316A10083121B
:100440008A0101208A11031C402C8316A00083120C
:100450008A0101208A11031C402C8316AD008312EF
:100460008A0101208A11031C402C8316AE008312DE
:100470008A0101208A11031C402C8316A9008312D3
:100480008A0101208A11031C402C8316AA008312C2
:100490008A0101208A11031C402C8316AB0021081D
:1004A0008312A9000130B000B101A5013A308A01E0
:1004B00031208A11031C402C6400831623080A3C57
:1004C0008A11831203197D2A640083162308143CC1
:1004D0008A1183120319D62A6400831623081E3C4E
:1004E0008A11831203194B2B640083162308283CBE
:1004F0008A1183120319C02B08008A115024831615
:100500000A30A8008312831621088312F6008F2078
:1005100064007508003C8A1103199D2AC8308A01BD
:1005200044208316A80364002808003C8A11831223
:1005300003199D2AF5018A01832A75088316A700ED
:1005400083128A11D8248A119C247E308A012B20A0
:100550007E308A012B20640083162D08003C8A110E
:1005600083120319BA2A8316240883128A012B20C6
:100570008A11BD2A00308A012B2083162708831296
:100580008A012B20640083162D08003C8A118312F7
:100590000319D12A8316250883128A012B208A1178
:1005A000D42A00308A012B208A11432C8A1150242E
:1005B00083160A30A8008312831620088312F600DF
:1005C000BB2064007508003C8A110319F62AC83064
:1005D0008A0144208316A80364002808003C8A117D
:1005E00083120319F62AF5018A01DC2A750883169D
:1005F000A60083128A11D8248A119C247E308A0195
:100600002B207E308A012B2083160130AC00831210
:10061000640083162C0820028A118312031C202BED
:1006200083162C083A3E840083120008B80038086C
:100630008A012B208316AC0A8A118312031D082B12
:10064000640083162D08003C8A11831203192F2B96
:100650008316240883128A012B208A11322B003042
:100660008A012B20640083162D08003C8A11831216
:100670000319412B8316250883128A012B208A1126
:10068000442B00308A012B208316260883128A010E
:100690002B208A11432C8A11502483160A30A8007B
:1006A0008312831620088312F600D4206400750894
:1006B000003C8A1103196B2BC8308A014420831631
:1006C000A80364002808003C8A11831203196B2BCD
:1006D000F5018A01512B75088316A60083128A1131
:1006E000D8248A119C247E308A012B207E308A01F6
:1006F0002B2083160130AC008312640083162C0873
:1007000020028A118312031C952B83162C083A3E73
:10071000840083120008B80038088A012B20831651
:10072000AC0A8A118312031D7D2B640083162D08E9
:10073000003C8A1183120319A42B83162408831208
:100740008A012B208A11A72B00308A012B208316C7
:10075000260883128A012B20640083162D08003C92
:100760008A1183120319BB2B8316250883128A0171
:100770002B208A11BE2B00308A012B208A11432C9A
:100780007E308A012B207E308A012B2052308A0154
:100790002B2053308A012B2032308A012B2033301A
:1007A0008A012B2032308A012B202D308A012B2008
:1007B0004B308A012B206F308A012B206E308A014A
:1007C0002B2076308A012B2065308A012B20723055
:1007D0008A012B2074308A012B2065308A012B205E
:1007E00072308A012B2020308A012B2056308A015A
:1007F0002B2030308A012B202E308A012B203530DF
:100800008A012B2068308A012B2020308A012B207E
:1008100044308A012B204C308A012B2031308A0150
:100820002B204D308A012B2046308A012B204B3063
:100830008A012B2020308A012B2030308A012B2086
:1008400035308A012B202F308A012B2032308A014B
:100850002B2030308A012B2031308A012B20303080
:100860008A012B2020308A012B2000308A012B2086
:1008700000308A012B2000308A012B208A11432C62
:1008800009308A012B204F308A012B204B308A01FE
:100890002B200D308A012B200A308A012B200800E2
:1008A000640083162D08003C8A11831203199B2CC7
:1008B0003A088316AF0083123B088316B0000A3053
:1008C000A80083120230F60083162D088312BA00A6
:1008D000FF3083162E078312B800FF300318013E45
:1008E000B9000130A00038088A016820BB008F20C1
:1008F00064007508003C8A1103198D2CC8308A01E8
:1009000044208316A80364002808003C8A1183123F
:1009100003198D2CF5018A01622C75088316A40039
:1009200083128A11D82483162F088312BA008316E3
:1009300030088312BB000800640083162D08003CB9
:100940008A1183120319D72C3A088316AF00831239
:100950003B088316B0000A30A80083120230F6006C
:1009600083162D088312BA00BB018F20640075081E
:10097000003C8A110319CB2CC8308A01442083160D
:10098000A80364002808003C8A1183120319CB2CA9
:10099000F5018A01AE2C75088316A5002F08831275
:1009A000BA00831630088312BB008A11D8240800CD
:1009B00064007508003C8A110319E02C8120F501C0
:0209C00008002D
:02400E006E3F03
:00000001FF
